:0C0000000C942B000C9400000C940000E9
:10000C000C9400000C9400000C9400000C94000064
:10001C000C9400000C9400000C9400000C94000054
:10002C000C9400000C9400000C9400000C94000044
:10003C000C9400000C9400000C9400000C94000034
:10004C000C9400000C9400000000F894EE27ECBB1C
:10005C00F1E0FBBFEBBFE5BFF8E1F1BDE1BD8DE029
:10006C00A2E0BB27ED938A95E9F780E098E0A0E643
:10007C00ED930197E9F7E4E5F0E085919591009710
:10008C0061F0A591B59105901590BF01F001059017
:10009C000D920197E1F7FB01F0CFEFE5EDBFE8E042
:1000AC00EEBFC0E6D2E00C945B00E0E0EBBBEABB39
:1000BC00E8BBE7BBE5BBE4BBE2BBE1BBE3BFE2BF34
:1000CC00ECBFEFBDEEBDEDBDECBDE7BDE6BDEBBDE0
:1000DC00EABDE9BDE8BDE2BDE5BDE4BDE3BDE5BFFC
:1000EC00E4BFE9BFE0E8E8B9E0E0E0BFFFCFFFCF55
:10300000310004B76C6F676F6F6F6F6F2E67696603
:103010005000007068746D6C6C6C6C6C2E68746D14
:10302000600000BC6A6176616161612E6A617661EF
:1031000047494638396132003200C40000020202E9
:103101002727281717184D4E4F666667393A3A0038
:103102003D9501449B01449D01439A064496134B0D
:10310300983467A6295EA41B529B4A76AD5E84B4AD
:103104006D91BC7598C28C8D8DABACAC8DABCCCDB8
:10310500CFD0C2D1E1DBE5EEFFFFFFFEFEFEFAFB0D
:10310600FCF3F6F7E7EBEDB1C3D47878782C000042
:103107000000320032000008FE0033081C485083DC
:10310800860C1D1E18389000C18187070C3460E0BA
:10310900C04002860E1B2A90B0C1E0418220430ACA
:10310A0034885021C4871A2B605809C1E2818C087F
:10310B00101888B021C34791386D965CF812630292
:10310C000315383C58F040C203050E1D429CD931C2
:10310D00A7D3842E21C64CB0A0830703061874C024
:10310E00C0E062CFA5349D16240955A9D4880F3688
:10310F006068E0A081070C48BD9E8C1896644EB293
:1031100026BF42BCB8404204030F3070A860C0EC28
:10311100DE974C6DDE0C79102AC6B94A255EF02087
:10311200A14306093C4F2A7598787148C72F0DA321
:103113004CF0B34105CA112A54941B9AE145031C90
:10311400411EFC083AA6DE040A1AE8D6DDB6EDEE36
:1031150006A4CD1AEE3C5B43CDB27AF72EF0C0A1E2
:10311600B9F3E7CE09CFDD2BB3AEE29D176D9FA4C1
:10311700EA412C41C20DE7FE36AC5ED3F8CEA4A23D
:10311800B92BF6C8BEFD41E99A4F326D9C57BBF2F8
:10311900EE7675E224093E3E58B579F967C0723AF0
:10311A0079769740D289D6136C153DA4A07A4D7959
:10311B00571082162918135218A547A0471232963A
:10311C00017C67E965DF430376D7A177FD399851C8
:10311D00760EDE9701071D40D75C8C33C268634184
:10311E003756A00064D3C9078140130420E49043BE
:10311F005230C004055050809003703010064B5A47
:1031200090C106C025D72389110059400102002013
:10312100C096000010E407014C10669826666066A0
:10312200014E72C0C0420AF668C08F0675F40100F3
:103123000468C041010050600106167800400003A6
:1031240000F0814D1B143A81406EC279E55C73EA6C
:1031250097C19D044CC92705035930A899013889D1
:1031260081000248F9E29B569266AAA991DA45A95E
:10312700A57D663AA805FF0100D09D99037CC4419F
:1031280003169D4ADA6FBC4A20E9AA1B5CEA6AA723
:10312900771E5A28A6026DF000AFBBC9E8DC064D30
:10312A001D04ACB00269DAA9A60558204000960D24
:10312B00E46C7310842BAEB815E437AD98035130B3
:10312C006807C1E28927411B4830EEB858D56B2F90
:10312D009D1FADAAA69713584041AC79EE8B264151
:10312E00B7DA6BEF95A9EAA42F07859E094001181F
:10312F0054DB259B04931AE7740957EBE7401B50B8
:10313000F001011F50E0E4481E6C5CB1A38F2EF536
:1031310063061E7FE0F2CB30C72CF3CB52BAC962D3
:10313200CA58DAB4D54A3CF7ECF3CF3D3BB981C566
:10313300571A964003119F28E1050BB0B6577090BC
:103134003210F162C64DF081BF14644DC104FD7AB2
:103135007881034EB7B899665959B698921F17D03A
:103136006F010314404001DD12F475665271161ECC
:103137008F594D9D6E99FE162499C10003189BA6C1
:10313800405FDF1D1F500DF6289356FA716064DB5F
:1031390098026E2CB284273EDDE219CC8DC0CD4BAE
:10313A00493DA59A6B177035A104F4AD77E1217664
:10313B008EC1417333D45AE76663D076E8216FB9F9
:10313C0068E574ABB8F8D4AC83BD396B3195CD6808
:10313D00B730DAC4414DB83B6D5BDEEBF57E51D84F
:10313E001131EE9DE69747CFFB75995BAE1D670C7F
:10313F0048E0FDF7E07B1F81E5187B6E60E5CFBFB0
:10314000FED24F06B71F15643F797E60E130B96E3D
:10314100D1FDB9E6FF934C9071AFF77ECEDB5CE722
:10314200181081898C0F300C60C0031C7094A10888
:10314300C77AD81309875A179A9954A00210C0A0B6
:10314400041670C10E62D0030E209BF9F22316EA16
:10314500FD445E12A8C0067524010FA8B00211281F
:103146008AEF48243FA5F58E27734A4D0452D312C1
:10314700F17DD001E33FF30AF39436921B32640119
:103148000A005B1249E3002422518948D99DA44E04
:103149003441B03DEF8A53998A545E33422216F1D5
:10314A00201ED891599E87801DB94E29A459C005C1
:10314B002228928000003B000000000000000000DD
:105000003C48544D4C3E0D0A3C424F445920626787
:10500100636F6C6F723D234330433043303E0D0A72
:105002003C68333E0D0A48544C20427261756E6111
:1050030075202121210D0A3C703E200D0A3C2F689A
:10500400333E200D0A4772FCDF6520766F6E204D1B
:10500500616E75656C264D617474686961730D0A0E
:105006003C2F424F44593E0D0A3C2F48544D4C3ECE
:105007000000000000000000000000000000000099
:10600000636C617373206170706C6574207B0D0A22
:1060010020207075626C6963207374617469632008
:10600200766F6964206D61696E28537472696E6778
:106003005B5D206172677329207B0D0A20202020AD
:10600400537472696E67206E616D65203D20224A6B
:106005006F686E223B0D0A2020202053797374653A
:106006006D2E6F75742E7072696E746C6E286E616B
:106007006D65293B0D0A2020202053797374656D37
:106008002E6F75742E7072696E746C6E286E616D69
:1060090065293B0D0A2020202053797374656D2E74
:10600A006F75742E7072696E746C6E286E616D6530
:10600B00293B0D0A20207D0D0A7D0D0A00000000A2
:00000001FF
